:0A00000075817F7401F58F02000E78
:10000B000208C275F15490000074F2F0A37407F06B
:10001B0090000274F2F0A37407F090000474F2F0F5
:10002B00A37407F012013FC209120FD4C2B6C2B5B6
:10003B00C2B71210B11210E2121113D2B6D2B5D24E
:10004B00B7C215C216C2177590FB75A0FFD2B4C20A
:10005B000FC212C210C213C211C214C200C202C21A
:10006B0004C201C203C205C206C207C208C209C24A
:10007B000AC20BD227D228D229C22DC22EC22FC21E
:10008B003FC240C241D221D222D223C23CC23DC286
:10009B003ED218D219D21A12012B120890D22AD2A0
:1000AB002BD22C7565C87567C87569C8755C647586
:1000BB005F80755D64756080755E64756180754287
:1000CB0000754300753A00753B0012048F1204C78C
:1000DB001204FF85424485434512053F12012B1242
:1000EB00012B12012B12114412033D12034F120369
:1000FB006112048F1204C71204FF1204AB1204E343
:10010B0012027712029E1202C512053F12056A12E5
:10011B0005950200F0783279FF0000D9FCD8F8225F
:10012B00786479FF0000D9FCD8F822781E7996D92B
:10013B00FED8FA22C2B6D2B5D2B712012B12012BBE
:10014B00C2B6C2B5D2B712012B12012BC2B6C2B5C1
:10015B00C2B712012B12012B12012B12012BC2B6AB
:10016B00C2B5D2B712012B12012BC2B6D2B5D2B780
:10017B0012012B12012BD2B6D2B5D2B712012B1210
:10018B00012B12012B12012B22E627F5290809E678
:10019B0037F52A782922C3E697F5290809E697F55A
:1001AB002A7829228629872B0809862A872C12026E
:1001BB0034782E22862E08862F08863008863187C3
:1001CB002B09872C1201D7782979302275320075CB
:1001DB0033101202191201EA12020DD533F422C3A5
:1001EB00E530952BE531952CE5329400500122E555
:1001FB0030952BF530E531952CF531E5329400F542
:10020B003222B3E52933F529E52A33F52A22C3E552
:10021B002E33F52EE52F33F52FE53033F530E53161
:10022B0033F531E53233F53222E529852BF0A4F590
:10023B002E85F02FE52A852CF0A4F53085F031E5DD
:10024B002A852BF0A4252FF52FE53035F0F530E579
:0F025B00313400F531E529852CF0A4252FF52F3E
:10026A00E53035F0F530E5313400F53122120A393E
:10027A00200C0122C20C30000C1205C01205E91232
:10028A00060CD2122212061C12062E120657D20F82
:10029A001203D122120A8D200D0122C20D30020C46
:1002AA0012066F1206981206BBD213221206CB123E
:1002BA0006DD120706D21012041422120AE1200ED9
:1002CA000122C20E30040C12071E12074712076AD7
:1002DA00D2142212077A12078C1207B5D21112040D
:1002EA00542230410122208110200110B200D20193
:1002FA00200005C218D2242222C201222230410142
:10030A0022208010200310B202D203200205C21953
:10031A00D2252222C203222230410122209010201B
:10032A000510B204D205200405C21AD2262222C21E
:10033A000522223000012220A708203C07D23CD205
:10034A001222C23C223002012220A708203D07D2F5
:10035A003DD21322C23D223004012220A708203EAA
:10036A0007D23ED21422C23E223084102009102025
:10037A002D05D218D20922D209C22D22C20922225F
:10038A00308510200A10202E05D219D20A22D20A4C
:10039A00C22E22C20A2222308210200B10202F05E0
:1003AA00D21AD20B22D20BC22F22C20B22222086B1
:1003BA0012200612B221D206D22DC21BC21CC23092
:1003CA00C23122C2062222201817C215C2B6202123
:1003DA0008120B568844894522120BCB884489455A
:1003EA0022855C5FC215D2B6A842A94388448945D2
:1003FA0022208712200712B222D207D22EC21DC291
:10040A001EC232C23322C2072222201917C216C2C2
:10041A00B5202208120C788846894722120CED88EA
:10042A0046894722C216D2B5A83CA93D88468947C3
:10043A0022208312200812B223D208D22FC21FC24E
:01044A002091
:10044B00C234C23522C2082222201A17C217C2B7E1
:10045B00202308120D9A8848894922120E0F8848CA
:10046B00894922C217D2B7A83EA93F884889492299
:10047B007A0FC294D2A2A2A133C933C9C2A2DAF2B3
:10048B00F8D29422D2947A0574E0C2A2C294339229
:10049B00A0D2A2DAF512047B8840894153410F2286
:1004AB00D2947A0574E8C2A2C2943392A0D2A2DA93
:1004BB00F512047B883C893D533D0F22D2947A057B
:1004CB0074F0C2A2C2943392A0D2A2DAF512047BCA
:1004DB00883A893B533B0F22D2947A0574F8C2A217
:1004EB00C2943392A0D2A2DAF512047B883E893FE4
:1004FB00533F0F22853A34853B3578348540388518
:10050B004139793812019486F008E6120EECF54366
:10051B0085F042228540348541357834853A3885DB
:10052B003B3979381201A186F008E6120EF9F54332
:10053B0085F04222A844A945D295D2A4E944707A09
:10054B0008C2A3C296339297D2A3DAF57A08E8C20F
:10055B00A3C296339297D2A3DAF5C295D29622A86C
:10056B0046A947D295D2A4E944F07A08C2A3C29611
:10057B00339297D2A3DAF57A08E8C2A3C2963392E4
:10058B0097D2A3DAF5C295D29622A848A949D2955B
:10059B00D296E944707A08C2A3C2A4339297D2A32D
:1005AB00DAF57A08E8C2A3C2A4339297D2A3DAF59C
:1005BB00C295D2A422200F0122D215C20FC21BC298
:1005CB001CC230C231755C64755F80120B359000B4
:1005DB0000858250858351754AFF754B14228550D7
:1005EB0082855183A943120833A3A842120843A35F
:1005FB00858250858351855056855157884489454E
:10060B0022D54A0C754AFFD54B06C200D22AC21816
:10061B002220120122C21290000085825085835144
:10062B00D22A22302A1D85508285518312086EA34F
:10063B0012087FA385825085835188718972886BDC
:10064B00896C22A86BA96C8871897222E556B582D8
:10065B0012E557B5830D302408D21212061CD22A8C
:10066B0022C22A2220100122D216C210C21DC21E83
:10067B00C232C233755D64756080120B4090283CAA
:10068B00858252858353754CFF754D14228552829A
:0B069B00855383A93D120833A3A83C3F
:1006A600120843A385825285835385525885535930
:1006B6008846894722D54C0C754CFFD54D06C2029B
:1006C600D22BC2192220130122C21390283C858204
:1006D60052858353D22B22302B1D8552828553831C
:1006E60012086EA312087FA38582528583538871F0
:1006F6008972886D896E22A86DA96E8871897222A9
:10070600E558B58212E559B5830D302508D2131286
:1007160006CBD22B22C22B2220110122D217C211C4
:10072600C21FC220C234C235755E64756180120B69
:100736004B905078858254858355754EFF754F14BE
:1007460022855482855583A93F120833A3A83E12F9
:100756000843A385825485835585545A85555B88FD
:1007660048894922D54E0C754EFFD54F06C204D294
:100776002CC21A2220140122C21490507885825469
:10078600858355D22C22302C1D85548285558312A3
:10079600086EA312087FA3858254858355887189C4
:1007A60072886F897022A86FA9708871897222E594
:1007B6005AB58212E55BB5830D302608D2141207AE
:1007C6007AD22C22C22C220000D2B30000000000F4
:1007D60000C2B3220000D2B3000000000000A2B4A1
:1007E600C2B3227E027A08EE3392B1FE1207CDDA48
:1007F600F622AE837A08EE3392B1FE1207CDDAF610
:10080600AE827A08EE3392B1FE1207CDDAF622E90D
:10081600FE7A08EE3392B1FE1207CDDAF622E8FE32
:100826007A08EE3392B1FE1207CDDAF622D2B2C2C0
:10083600B01207E91207F8120815D2B022D2B2C2D6
:10084600B01207E91207F8120824D2B0227E037A02
:1008560008EE3392B1FE1207CDDAF6227A081207B5
:10086600DAEE33FEDAF8F422D2B2C2B0120853122C
:1008760007F8120862F9D2B022D2B2C2B0120853F7
:100886001207F8120862F8D2B0227587907589228D
:10089600759850758C38758A38C0D043D00878144E
:1008A60079647A197B327C197D02D0D07565007522
:1008B6006700756900D28CD2A9D2AF22C0E0C0D041
:1008C60043D008DD557D02D83F7819120935120943
:1008D6007E1209C712037312038A1203A11202ECD5
:1008E6001203071203220565E565120EBCF56505C0
:1008F60067E567120EBCF5670569E569120EBCF57A
:1009060069DC057C19120925D904A95CD20CDA0424
:10091600AA5DD20DDB04AB5ED20ED0D0D0E0323071
:100926001502B2B6301602B2B5301702B2B722308F
:100936000001222084041203B82220861C200627E8
:10094600D212D206D227756500756600D224C21867
:0D095600C21BC21CC230C23122C2063027B3
:1009630009C22785656612096E2222E566B428034B
:1009730002097B5003C22422D22422300201222006
:1009830085041203FB2220871C200727D213D207DA
:10099300D228756700756800D225C219C21DC21E10
:1009A300C232C23322C207302809C22885676812BF
:1009B30009B72222E568B428030209C45003C225FB
:1009C30022D225223004012220820412043B222059
:1009D300831C200827D214D208D229756900756AAE
:1009E30000D226C21AC21FC220C234C23522C20894
:1009F300302909C22985696A120A002222E56AB4EC
:100A03002803020A0D5003C22622D22622E582C4FD
:100A1300540FF9E583C46922B48003020A2E500BF4
:100A230075F0038475F002A424102275F005847513
:100A3300F003A424322230000122301801222021A5
:100A43000122853A82853B83120A10301B0EF55F23
:100A5300F4120A1B120ED9F55CC21C22201C10D200
:100A63001CB55F03D21B225003C23922D239222084
:100A7300390CB55F03D21B22500122D21B22B55F72
:100A830003D21B225003D21B22223002012230192F
:100A9300012220220122853C82853D83120A1030E7
:100AA3001D0EF560F4120A1B120ED9F55DC21E224B
:100AB300201E10D21EB56003D21D225003C23A225B
:100AC300D23A22203A0CB56003D21D22500122D221
:100AD3001D22B56003D21D225003D21D22223004F1
:100AE3000122301A012220230122853E82853F8381
:100AF300120A10301F0EF561F4120A1B120ED9F5FB
:100B03005EC22022202010D220B56103D21F2250C2
:100B130003C23B22D23B22203B0CB56103D21F22EE
:100B2300500122D21F22B56103D21F225003D21FCC
:100B3300222290000074F2F0A37407F022900002C6
:100B430074F2F0A37407F02290000474F2F0A3741B
:100B530007F02230210122853A82853B83120A1055
:100B630030301CF56275F080846006120C3C020B79
:100B730077120C00900000E53AF0A3E53BF0222049
:100B83003119D231B56206D230120BCB225006C2D4
:100B930036120BCB22D236120BCB22203615B5627E
:100BA30006D230120BCB225004120BCB22D23012BE
:100BB3000BCB22B56206D230120BCB225006D230B9
:100BC300120BCB22120BCB22900000E0F582900097
:100BD30001E0F583120A1075F08084601090000024
:100BE300E0F534900001E0F535120C42229000004C
:100BF300E0F538900001E0F539120C0622853A3809
:100C0300853B397938753400753508753600753785
:100C13000078341201A18638088639793885713411
:100C230085723575360075370078341201A186F068
:100C330008E6120EF9F9A8F022853A34853B35759A
:100C430036007537007834753800753908793812ED
:100C530001A18634088635753600753700783485EA
:100C63007138857239793812019486F008E6120ECC
:100C7300ECF9A8F02230220122853C82853D8312C3
:100C83000A1030321CF56375F080846006120D5E25
:100C9300020C99120D22900002E53CF0A3E53DF011
:100CA30022203319D233B56306D232120CED22500F
:100CB30006C237120CED22D237120CED2220371563
:100CC300B56306D232120CED225004120CED22D27F
:100CD30032120CED22B56306D232120CED2250060D
:100CE300D232120CED22120CED22900002E0F582BA
:100CF300900003E0F583120A1075F0808460109071
:100D03000002E0F534900003E0F535120D64229003
:100D13000002E0F538900003E0F539120D28228532
:100D23003C38853D3979387534007535087536009A
:100D330075370078341201A18638088639793885E9
:100D4300713485723575360075370078341201A118
:100D530086F008E6120EF9F9A8F022853C34853DA9
:100D6300357536007537007834753800753908796C
:100D7300381201A186340886357536007537007838
:100D830034857138857239793812019486F008E612
:100D9300120EECF9A8F02230230122853E82853F12
:100DA30083120A1030341CF56475F08084600612D7
:100DB3000E80020DBB120E44900004E53EF0A3E545
:100DC3003FF022203519D235B56406D234120E0F06
:100DD300225006C238120E0F22D238120E0F2220D2
:070DE3003815B56406D23497
:100DEA00120E0F225004120E0F22D234120E0F22AC
:100DFA00B56406D234120E0F225006D234120E0FE8
:100E0A0022120E0F22900004E0F582900005E0F510
:100E1A0083120A1075F080846010900004E0F534A3
:100E2A00900005E0F535120E8622900004E0F538B0
:100E3A00900005E0F539120E4A22853E38853F3981
:100E4A007938753400753508753600753700783489
:100E5A001201A18638088639793885713485723548
:100E6A0075360075370078341201A186F008E6124B
:100E7A000EF9F9A8F022853E34853F35753600759E
:100E8A003700783475380075390879381201A18627
:100E9A00340886357536007537007834857138859B
:100EAA007239793812019486F008E6120EECF9A824
:100EBA00F022B4C8012250012274C822B43201229D
:100ECA005003743222B4C8012250012274C822B4D9
:100EDA001001225003741022B4C801225001227456
:100EEA00C822B40F0122500122740F75F0FF22B4F8
:100EFA000F0122500122740075F00022120FA6740D
:100F0A00A0F9120F73120FC2E573F9120F73120FC1
:100F1A00C2E574F9120F73120FC2120FA674A1F967
:100F2A00120F73120FC2120F66120FC2120F9822FB
:100F3A00E9FA120FA674A0F9120F73120FC2E57321
:100F4A00F9120F73120FC2E574F9120F73120FC25E
:100F5A00EAF9120F73120FC2120F9822D29178086F
:100F6A00120FC8E933F9D8F8227808E9339291F9CF
:100F7A00120FC8D8F6227B80DB02800E120FA674ED
:100F8A00A0F9120F73120FC240EE120F9822C291EB
:100F9A0000D292000000000000D29122D29100D229
:100FAA0092000000000000C291000000000000C290
:100FBA009222C291120FC822D291120FC8220000A7
:100FCA00D292000000A291C292222084292009FA1A
:100FDA00C2B6C2B5C2B712100312103D1210771270
:100FEA00012B12012B12012B12012BD2B6D2B5D230
:100FFA00B7D209020FD4C20922900000754A1975A6
:10100A004B018583738582747900120F3A120F801F
:10101A00A38583738582747900120F3A120F80A315
:10102A00858256858357D54AD9754A19D54BD31225
:10103A0011DC2290283C754C19754D018583738506
:10104A0082747900120F3A120F80A3858373858206
:10105A00747900120F3A120F80A38582588583593A
:10106A00D54CD9754C19D54DD31211FD2290507813
:10107A00754E19754F018583738582747900120F35
:10108A003A120F80A38583738582747900120F3A0E
:10109A00120F80A385825A85835BD54ED9754E1966
:1010AA00D54FD312121E2212123F9000008583736D
:1010BA00858274120F06E9F9120833A385837385B2
:1010CA008274120F06E9F8120843A3E556B582DDC9
:1010DA00E557B583D8D22A2212125A90283C858322
:1010EA0073858274120F06E9F9120833A385837394
:1010FA00858274120F06E9F8120843A3E558B582EF
:10110A00DDE559B583D8D22B221212759050788515
:10111A008373858274120F06E9F9120833A3858353
:10112A0073858274120F06E9F8120843A3E55AB5CB
:10113A0082DDE55BB583D8D22C2220A524201801B4
:10114A002220190122201A01223000012230020134
:0E115A002230040122D241203F1DD23FD2405C
:10116800C24222C23F304014C2401211C03081FD39
:101178003080FA3090F7C2412212118522304201A4
:101188002220810FC2B612012BD215121290D2B6AC
:10119800D2422220800FC2B512012BD2161212C5DC
:1011A800D2B5D2422220900FC2B712012BD2171209
:1011B80012FAD2B7D242222230420122D215D216D6
:1011C800D2171212901212C51212FAD2B6D2B5D292
:1011D800B7D24222907850A95685837385827412BB
:1011E8000F3A120F80A3A957858373858274120F53
:1011F8003A120F8022907852A95885837385827499
:10120800120F3A120F80A3A959858373858274122D
:101218000F3A120F8022907854A95A8583738582D9
:1012280074120F3A120F80A3A95B858373858274A9
:10123800120F3A120F80229078508583738582743A
:10124800120F068956A3858373858274120F068947
:101258005722907852858373858274120F068958B5
:10126800A3858373858274120F0689592290785456
:10127800858373858274120F06895AA385837385C3
:101288008274120F06895B221211DC90000012088A
:101298006E858373858274E9F9120F3A120F80A361
:1012A80012087F858373858274E8F9120F3A120F4A
:1012B80080A3E556B582D7E557B583D2221211FD32
:1012C80090283C12086E858373858274E9F9120FA1
:1012D8003A120F80A312087F858373858274E8F918
:1012E800120F3A120F80A3E558B582D7E559B58396
:1012F800D22212121E90507812086E85837385824E
:1013080074E9F9120F3A120F80A312087F858373CC
:10131800858274E8F9120F3A120F80A3E55AB58254
:10132800D7E55BB583D222464C414D45204B4E4F05
:10133800425245434F524445522D43332D4D4F445D
:10134800554C45204555524F205241434B20564558
:101358005253494F4E202D203230313120564552BC
:1013680053494F4E20312E3031202863296279208D
:06137800616D70657265F5
:00000001FF
